:020000040000FA
:0400000085284430DB
:08000800A000030EA100831209
:100010000C1C2328DD1B23288E015C1C15285C107A
:1000200050088F005D0985051B285C1451088F005E
:100030005D088504DC170C108B180828210E83003E
:10004000A00E200E090005192B2883160117831214
:10005000B23081005D288316011383120B193728F3
:10006000AE17280A03192E17AE1948285628AE13C2
:10007000AE1945282E1F5628AE1A5628A701A601EC
:10008000A501A801AE01AE165D28F030AE055D28D1
:100090002D152E13AE122708AB002608AA0025083E
:1000A000A9002808AC00F030AE055D282E0DA80D83
:1000B000A50DA60DA70DAE1AAE0A8B100B11210EC1
:0800C0008300A00E200E0900D0
:06010A002030840080019A
:10011000840A80300402031C8728772283160C305F
:10012000850587018312850187010730990000301A
:100130009A00103083168E008312603083168F0071
:1001400083120030831691009F008312C8308316FB
:100150008100831201309000A63096001830910083
:100160008030970007309300013083168C00831293
:1001700010308B00362381018E018F010B118B1003
:100180000B108C010B178B17D9202D19DB20701841
:10019000C4284722B30BD728031085190314BA0DBE
:1001A000F0303A020319BF21F308031991261C24E9
:1001B000C4286400080045257018080029083F3C41
:1001C0000319EA282B082A0629062C02031D2D11E3
:1001D000031D08002D110130B7008B1320303707A5
:1001E00083169B001C141A088312A40010303707D2
:1001F00083169B001C141A088312A30000303707D3
:1002000083169B001C141A088312A2008B17240863
:100210002B02031DB92923082A02031DB929013025
:100220003702031D492929083F3C03193329A91B1B
:100230001F29291F1F2929081F39AF00AF17403078
:100240002906E039031D29293F1F29293F13AD172E
:10025000372960302906E039031D37293F1B37292C
:100260003F17AD173729AC1F3F13AC1B3F1780302A
:100270002906F039031D4029BF1F4029BF13AD17C0
:1002800090302906F039031D4929BF1B4929BF17A2
:10029000AD17A91FB929291BB92922082906F03948
:1002A000A91EE039031DB929220829050F390319B0
:1002B000862901303702031D62293E1862293E1447
:1002C000AD17A62202303702031D6B29BE186B2919
:1002D000BE14AD17C12203303702031D74293E1925
:1002E00074293E15AD17DC2204303702031D7D2929
:1002F000BE197D29BE15AD17F72205303702031D43
:1003000086293E1A86293E16AD1712232909220591
:100310000F390319B92901303702031D94293E1CF6
:1003200094293E10AD171C2302303702031D9D296E
:10033000BE1C9D29BE10AD17202303303702031DBC
:10034000A6293E1DA6293E11AD17242304303702ED
:10035000031DAF29BE1DAF29BE11AD1728230530DF
:100360003702031DB8293E1EB8293E12AD172C23B3
:10037000B929B70A0630370203180800ED2808002B
:100380000B13DD17B601B3019630B4000130B50090
:100390000130B70085018701AD132C22D920B30BA2
:1003A000EB29031085190314BA0DF0303A02031932
:1003B0001A2AB41F8501B41F8701B40BEB29370833
:1003C000B6080319B6000319E929FF308500870034
:1003D000B6039630B4002D1DCE292D11A91FCE29AC
:1003E000291BCE29A91E29120F3029050319CE2950
:1003F000B9012918B90AA918B90A2919B90AA919F4
:10040000B90AB918CE293919CE298B1320303707EC
:10041000BC002B08BB00572210303707BC002A084D
:10042000BB00572200303707BC002908BB00572209
:100430008B17262285018701B70AB60106303702DD
:10044000031CCE290B17DD133623080005303702B5
:1004500003190800850187011430B90033308F1F5C
:1004600085008F1B8501D9202D1D2E2A2D11290ACB
:1004700003193E2AA91F2E2A291B2E2A0F302905CF
:10048000031D2C2AB90B2E2A8501870108005C1C4C
:100490000800AD1F0800AD131030BC003E08BB00C3
:1004A00057223030BC003F08BB00572208003C08F0
:1004B0008B1383169B001C141A0883128B173B02A4
:1004C000031908008B133B0883161C159A0083122E
:1004D0003C0883169B0055309D00AA309D009C145B
:1004E00064009C18702A1C1183128B1708000A30B4
:1004F000DE007D30DF00831600309B001C141A08DC
:100500008312BD00831610309B001C141A0883123E
:10051000BE00831630309B001C141A088312BF00E3
:100520006230F100E0267208C0006330F100E0267E
:10053000720840020319F0166D30F100E0267208CF
:10054000E1006118BE016118BF0108008B1383161A
:1005500073309B001C141A088312C1008B175210B1
:100560000E303E05031D08008B1383166F309B0071
:100570001C141A088312C5008B178E018F010C10F2
:1005800008008B13831673309B001C141A08831207
:10059000C2008B17D2100D303E05031D08008B13CF
:1005A00083166F309B001C141A088312C5008B172A
:1005B0008E018F010C1008008B13831673309B0083
:1005C0001C141A088312C3008B1752110B303E05FE
:1005D000031D08008B1383166F309B001C141A0830
:1005E0008312C5008B178E018F010C1008008B132E
:1005F000831673309B001C141A088312C4008B17D7
:10060000521207303E05031D08008B1383166F300E
:100610009B001C141A088312C5008B178E018F01D2
:100620000C1008008B13831671309B001C141A08E1
:100630008312CF008B170800E61F8512DD12080019
:10064000E71F05125D120800E81F8510DD10080085
:10065000E91F05105D1008008B13831672309B0094
:100660001C141A088312CF008B170800C101C201A5
:10067000C301C4013E1E2C2B122B08005308C6399F
:10068000031908005418DD12D4185D125419DD1036
:10069000D4195D10D31F542B3F1F512B531F542BC4
:1006A0007A2B531B542B7A2B5319622BD3185B2BA9
:1006B000BF1B6F2B7A2B54083E0503197A2BDC18CD
:1006C0006F2B7A2B54083E050319782B5C1D7A2B6F
:1006D0005B085405031D08005408DB046F2B5418F5
:1006E0008516D418051654198514D4190514080054
:1006F0005408DB0454188512D418051254198510B7
:10070000D41905100800701E08008B1383162008EA
:100710008400000883128B1795008B138316A00AA0
:10072000AB302002A1300318A00083128B17080001
:100730006430F100E0267208F500E01EF501653036
:10074000E01E6030F100E0267208F6008B1383167D
:10075000A130A0007730A100AD30A20083128B172A
:10076000AD30761CAF30F61C40388B138316A300D7
:1007700083128B17AD30761DAF30F61D40388B13CA
:100780008316A40083128B17AD30761EAF30F61E91
:1007900040388B138316A50083128B17AD30761F5C
:1007A000AF30F61F40388B138316A60083128B17C9
:1007B000AD30751CAF30F51C40388B138316A70085
:1007C00083128B17AD30751DAF30F51D40388B137C
:1007D0008316A80083128B17AD30751EAF30F51E3F
:1007E00040388B138316A90083128B178330F100D6
:1007F000E0267203C000AD30401CAF30C01C403852
:100800008B138316AA0083128B178B13831623096D
:10081000A2062409A2062509A2062609A20627097E
:10082000A2062809A2062909A2062A09A206AD30B5
:10083000A20483128B1708004F08FF3CD100F03050
:100840004F07D0008323D40154146608D3003E23FD
:10085000D401D4146708D3003E23D401541568088A
:10086000D3003E23D401D4156908D3003E23F224DB
:100870003125C5080319452CDC1F0800DC13DF0BEC
:1008800008007D30DF00C50308006608C639031D77
:100890004D2C3E1CDD123E18DD166708C639031DBF
:1008A000552CBE1C5D12BE185D166808C639031DA6
:1008B0005D2C3E1DDD103E19DD146908C639031D8F
:1008C000652CBE1D5D10BE195D14DE0B08000A30DC
:1008D000DE00521C8512D21C0512521D8510D21D3D
:1008E00005108324661896246718AA246818BC2467
:1008F0006918CE24661C5214671CD214681C521549
:10090000691CD21508004B08CA00E024CB004C0833
:10091000CA00E024CC004D08CA004B1CE024CD00E6
:100920004E08CA00CB1CE024CE000800C108031901
:10093000521403190800C60B0800CB1BC1034B0857
:10094000C600CB1852144B195214CB1E5214CB1D97
:1009500052100800C2080319D21403190800C70B6B
:100960000800CC1BC2034C08C700CC1AD2144C1D83
:10097000D2144C1FD2100800C308031952150319D2
:100980000800C80B0800CD1BC3034D08C8004D1A52
:1009900052154D1F5215CD1D52110800C4080319E0
:1009A000D21503190800C90B0800CE1BC4034E085A
:1009B000C9004E1AD215CE1FD215CE1DD211080075
:1009C000C001CA080319CA034A184014CA1A4014BD
:1009D0004008C0014A1C4014CA1E4014C005C00C87
:1009E0004A0C0800D60B0800AF1F0E2D03102F1A5B
:1009F0000314AF0D1F30AF05AF1358082F02031CAF
:100A0000072D03190E2D2F08D800D5000E2D2F0805
:100A1000D80065080319D5076308D700580864078C
:100A200055020318222DDC10E6188512E71805126E
:100A3000E8188510E91805105808013E55020318FA
:100A40002B2D0800DC14E6188516E7180516E818A3
:100A50008514E9180514D70B08006308D700D503DF
:100A60000800DA0B0800D90B08008B1383167A30C4
:100A70009B001C141A088312D9008B175C1D422D91
:100A80005C110800DB015C1508007018572D2A085E
:100A900003194C2DF30108002908031D08002D112E
:100AA000F30A06307302031C080070140800850165
:100AB00087012D112B082A0629020319662D2B0800
:100AC0002A0629062C020319662D08007C302B0605
:100AD000FC390319E02D701178302B06FC3903190D
:100AE0007E2D74302B06FC390319C72D2B080319F2
:100AF00008007010F3017012912608007608290290
:100B0000031908002908F600E0307606E039031DD5
:100B100008000130F6180430F50003107618F50DC2
:100B20007619F50EF825F201F019A32D8B13710833
:100B300083169B001C141A088312F2008B17403096
:100B4000F1080319F200761AB12DF01E08007208A0
:100B500075050319AE2DF6194A260800F61D4A261A
:100B60000800701F080007302A0203190800F61D4C
:100B7000BC2D7508F204BE2D7509F2058B137108A2
:100B8000BC007208BB0057228B174A260800F01ED3
:100B90000800F825F201F019DA2D8B13710883167D
:100BA0009B001C141A088312F2008B174030F108C6
:100BB0000319F20072082902031D08004A260800E2
:100BC00070190800F825701F0800F0190800F108D6
:100BD0000319EA2E07302A02031908008B13710843
:100BE000BC002908BB0057228B1770154A26080045
:100BF000F0157013F01A70172B180800AB180800C6
:100C0000F011AA0AF10108302A0203190800603025
:100C1000F10001302A0203190800F10A07302A0204
:100C200003190800F10A0F302A020319701703197B
:100C30000800F10A10302A0203190800F10A1130E5
:100C40002A0203190800F10A12302A0203190800C7
:100C5000F10AF10AF10A1D302A02031908003030A6
:100C6000F4006D30F10074082A0203190800F40A38
:100C70004130740269300319F4006B307402703033
:100C80000319F400A03074020319F01503190800C9
:100C9000F10A332EFF30850087003130900000309C
:100CA00083168C0083128E018E17FC308F000C107F
:100CB00064000C1C582E0C10850187010130900037
:100CC000013083168C00831208006830F100E026A2
:100CD0007208E0007A30F100E0267208D9007B301B
:100CE000F100E0267208E3007C30F100E026720893
:100CF000E4007D30F100E0267208E5006D30F1007F
:100D0000E0267208E10066308400A630F100E0269B
:100D100072088000F10A840A70300402031C872ED6
:100D20000800701A08007016652698236430F100D8
:100D3000E0267208F500E01EF5016530E01E603027
:100D4000F100E0267208F6000130F4007408103E4D
:100D5000F100E0267608F2020319B42E8B13BB00D3
:100D60007108BC0057228B177408203EF100E02662
:100D70007508F2020319C22E8B13BB007108BC0068
:100D800057228B179B307407F100E02672080F3949
:100D9000F8008027F7007408003EF100E02677088D
:100DA000F2020319D92E8B13BB007108BC00572225
:100DB0008B17F40A0B30740203190800A62E0800E2
:100DC0008B13710883169B001C141A088312F200FF
:100DD0008B170800F4016030F1008B137108831643
:100DE0009B001C141A088312F2008B177408F80079
:100DF000A027F2020319022F8B13BB007108BC005D
:100E000057228B17F40A5030740203194A2EF10A44
:020E1000ED2EC5
:100F000007308A0078088207903481348234843430
:100F10008834B134B234B434B834A134A234A434F3
:080F2000A834813481348134CE
:100F400007308A007808820703343E3401340134C4
:100F5000C034013400340034003400340034003430
:100F60000034003400340034003402340F340434CC
:100F7000FF34FF34FF34FF34FF34FF3405340434CE
:100F800004341034FF34FF34FF34FF34FF340134B1
:100F9000FF34FF34FF34FF34FF34FF34FF34FF34B9
:100FA000FF34FF34FF34FF34FF34FF34FF34FF34A9
:100FB000FF34FF34FF34FF34FF34FF34FF34FF3499
:100FC000013402340334043405340634073408345D
:100FD00009340A34013401348034C034013401341A
:0A0FE0000134013401340134FF3400
:084000000C00000006000200A4
:02400E00CC33B1
:1042000001008100820084008800B100B200B40087
:10421000B800A100A200A400A800FF00FF00FF005A
:104220000300030003000300030003000300030076
:1042300003000300030003000300FF00FF00FF0072
:10424000FF0000000000000000000000000000006F
:1042500000000000000000000000FF00FF00FF0061
:10426000FF00FF00FF00FF00FF00FF00FF00FF0056
:10427000FF00FF00FF00FF00FF00FF00FF00FF0046
:10428000FF00FF00FF00FF00FF00FF00FF00FF0036
:10429000FF00FF00FF00FF00FF00FF00FF00FF0026
:1042A000FF00FF00FF00FF00FF00FF00FF00FF0016
:1042B000FF00FF00FF00FF00FF00FF00FF00FF0006
:1042C00003003E0001000100C000010000000000EA
:1042D00000000000000000000000000000000000DE
:1042E000000002000F000400FF00FF00FF00FF00BD
:1042F000FF00FF000500040004001000FF00FF00A5
:10430000FF00FF00FF000100FF00FF00FF00FF00B3
:10431000FF00FF00FF00FF00FF00FF00FF00FF00A5
:10432000FF00FF00FF00FF00FF00FF00FF00FF0095
:10433000FF00FF00FF00FF00010002000300040077
:10434000050006000700080009000A00010001003E
:104350008000C00001000100010001000100010017
:10436000FF00FF00FF00FF00FF00FF00FF00FF0055
:10437000FF00FF00FF00FF00FF00FF00FF00FF0045
:10438000FF00FF00FF00FF00FF00FF00FF00FF0035
:10439000FF00FF00FF00FF00FF00FF00FF00FF0025
:1043A000FF00FF00FF00FF00FF00FF00FF00FF0015
:1043B000FF00FF00FF00FF00FF00FF00FF00FF0005
:1043C000FF00FF00FF00FF00FF00FF00FF00FF00F5
:1043D000FF00FF00FF00FF00FF00FF00FF00FF00E5
:1043E000AA00FF00FF00FF00FF00FF00FF00FF002A
:1043F000FF00FF00FF00FF00FF00FF00FF00FF00C5
:00000001FF
